:100000000C949A010C94C2010C94C2010C94C2018C
:100010000C94C2010C94C2010C94C2010C94C20154
:100020000C94C2010C94C2010C94B81A0C9484195B
:100030000C94C2010C94C2010C94C2010C94C20134
:100040000C94C2010C943D0A0C94C2010C94C201A0
:100050000C94C2010C94C2010C94C2010C94EE12D7
:100060000C94C2010C94C2010C94C2010C94C20104
:100070000C94C2010C94C2010C94C2010C94C201F4
:100080000C94C2010C94C2010C94C2010C94C201E4
:100090000C94010E0C94C2010C94C2010C94C20188
:1000A0000C94C2010C94C2010C94C20183099F09F3
:1000B000C3089F0934099F09A10850089F099F0997
:1000C0009F099F099F0967079F0936089F098808AC
:1000D00047144C1451145B146514AF14AF14AF14CF
:1000E0006F14791483148D149A14AF14A214D014BD
:1000F000D314C214C614CC14F414F414F414D71486
:10010000DB14DF14E514E914F414EF1407060504F6
:100110000100080A0B0C0D090000000200090F0085
:1001200000030401000C00000000000000000000BB
:100130000000000000000408020110408040102070
:10014000408040800802040180402010020110809D
:1001500010204040040404040403040502020202C7
:100160000403020202020606060606060404020250
:100170000204000000002300260029002C002F00AC
:1001800000000000250028002B002E003100000098
:100190000000240027002A002D003000080B000278
:1001A000020201000904000001020200000524000F
:1001B00010010524010101042402060524060001A2
:1001C0000705810310004009040100020A00000035
:1001D000070502024000000705830240000000C13D
:1001E0008081C112010002020000404123368000DC
:1001F000010102000112010002000000404123360B
:100200008000010102000141726475696E6F204C2B
:100210004C430041726475696E6F204C656F6E616E
:1002200072646F0004030904000000000000000075
:100230002A2B280000000000000000000000000041
:1002400000000000000000002C9EB4A0A1A2A43475
:10025000A6A7A5AE362D3738271E1F20212223241E
:100260002526B333B62EB7B89F8485868788898ABA
:100270008B8C8D8E8F909192939495969798999A56
:100280009B9C9D2F3130A3AD350405060708090A54
:100290000B0C0D0E0F101112131415161718191A36
:1002A0001B1C1DAFB1B0B500090402000103000022
:1002B00000092101010001226500070584034000B7
:1002C0000105010902A1010901A100850105091922
:1002D000012903150025019503750181029501751A
:1002E00005810305010930093109381581257F751C
:1002F0000895038106C0C005010906A10185020514
:100300000719E029E7150025017501950881029577
:1003100001750881039506750815002565050719FF
:100320000029658100C0CC061F0DDF12E3125016B4
:10033000B316AA1C11241FBECFEFDAE0DEBFCDBF7B
:1003400011E0A0E0B1E0E2E2FDE302C005900D9211
:10035000A43FB107D9F724E0A4EFB1E001C01D929A
:10036000A83BB207E1F713E0C4E3D3E004C022974F
:10037000FE010E94161DC632D107C9F70E94C3169E
:100380000C948F1E0C9400001F93CF93DF93162FB5
:10039000843008F06CC0982F990F990F990F985FCF
:1003A0009F3108F09EE1D82FDD0FDD0FDD0F8D2F7F
:1003B000C0E041E08917C8F4E82FF0E0DF01A05366
:1003C000BD4F2C91223070F4C42BEE0FFF1FE0576D
:1003D000FD4F21E030E0542F512311F420E030E0B4
:1003E00031832083440F8F5FE5CFC0FF05C0612FAD
:1003F00061708D2F0E942E15C1FF06C0612F6270A3
:1004000081E08D0F0E942E15C2FF06C0612F64701F
:1004100082E08D0F0E942E15C3FF06C0612F687009
:1004200083E08D0F0E942E15C4FF06C0612F6071FE
:1004300084E08D0F0E942E15C5FF06C0612F6072EB
:1004400085E08D0F0E942E15C6FF06C0612F6074D7
:1004500086E08D0F0E942E15C7FF09C0612F6078BE
:1004600087E08D0FDF91CF911F910C942E15DF91B6
:10047000CF911F9108950F931F93CF93DF93EB01BB
:100480008E3178F5082F10E0F801E053FD4F908190
:10049000933089F0943029F5F801ED5FFD4F20810C
:1004A00030E0C901880F991F820F931F8F5D9D4F08
:1004B0000E94DA0B0FC0833051F09BEF980F9230FF
:1004C00030F097EF980F933010F08D3019F4BE0193
:1004D0000E942114F801EE0FFF1FE057FD4FD1835A
:1004E000C083DF91CF911F910F910895CF93C82FB3
:1004F0008C3058F54091F6025091F70221E030E03F
:10050000082E02C0220F331F0A94E2F7672B49F42A
:1005100020953095242335233093F7022093F6025B
:1005200014C0242B352B3093F7022093F6028091D0
:10053000F40181110AC08C2F0E94F013AC016C2FC2
:100540008EED93E0CF910C94A910CF910895DB012B
:100550009A019091F5019C30D0F54091F601682FF9
:1005600070E0442369F0E42FF0E0EA50FE4F808110
:10057000FB01ED5FFD4F808341504093F60107C0C2
:10058000FB01ED5FFD4F90839F5F9093F501FB01B1
:10059000ED5FFD4F1A161B067CF41216130664F469
:1005A000408150E0CA01880F991F840F951FAD014B
:1005B0008F5D9D4F0C94150B208130E0C901880F91
:1005C000991F820F931F8F5D9D4F0C94930B68E1D1
:1005D00071E08EED93E00C943811CF93DF93C82F28
:1005E000D0E0CD5FDD4F288130E0C901880F991F31
:1005F000820F931F8F5D9D4F0E94990B8881909170
:10060000F501891306C0882379F081508093F501A4
:100610000BC0992349F0E091F601EF5FE093F601FA
:10062000F0E0EA50FE4F80838FEF8883DF91CF9117
:1006300008951F93CF93DF93162FC82FD0E0FE01AC
:10064000E453FD4F90811923C251DD4F411103C086
:100650009881911741F0412F50E0682F8EED93E083
:100660000E94C2101883DF91CF911F910895EF92DD
:10067000FF920F931F93CF93DF93E82E83E08E15A5
:1006800008F475C02E2D30E0F901EE50FD4F608367
:10069000672B09F46CC0F901E453FD4FF0800E2D77
:1006A000000F000F000FF0FE52C0802F0E94641553
:1006B000892B09F44CC011E0C02FD0E0F1FE07C037
:1006C00081E0800F0E946415892B09F042C0F2FE80
:1006D00006C082E0800F0E946415892BE1F5F3FECD
:1006E00006C083E0800F0E946415892BB1F5F4FEEB
:1006F00006C084E0800F0E946415892B81F5F5FE09
:1007000006C085E0800F0E946415892B51F5C83121
:10071000D10541F0F6FE06C086E0800F0E94641508
:10072000892B09F5679744F4F7FE06C087E0800F30
:100730000E946415892BC9F441E0612F8E2DDF9151
:10074000CF911F910F91FF90EF900C94190310E03F
:10075000B3CF1260BCCF1460C2CF1860C8CF106195
:10076000CECF1062D4CF1064DDCF1068E5CFDF911B
:10077000CF911F910F91FF90EF900895CF93DF934A
:100780008091F202882309F448C0D091CC02D0FFB6
:100790001DC180E00E946415892B09F417C1C1E0D6
:1007A000D1FF06C081E00E946415892B09F010C1B9
:1007B000D2FF06C082E00E946415892B09F00AC1AD
:1007C000D3FF06C083E00E946415892B09F004C1A1
:1007D000D4FF06C084E00E946415892B09F0FEC096
:1007E000D5FF06C085E00E946415892B09F0F8C08A
:1007F000D6FF06C086E00E946415892B09F0F2C07E
:10080000D7FF06C087E00E946415892B09F0ECC071
:1008100040E06C2F80E00E9419038091F30288234E
:1008200009F448C0D091CD02D0FFE0C088E00E941A
:100830006415892B09F4DAC0C1E0D1FF06C089E054
:100840000E946415892B09F0D3C0D2FF06C08AE04C
:100850000E946415892B09F0CDC0D3FF06C08BE040
:100860000E946415892B09F0C7C0D4FF06C08CE034
:100870000E946415892B09F0C1C0D5FF06C08DE028
:100880000E946415892B09F0BBC0D6FF06C08EE01C
:100890000E946415892B09F0B5C0D7FF06C08FE010
:1008A0000E946415892B09F0AFC040E06C2F81E0F5
:1008B0000E9419038091F402882309F448C0D09162
:1008C000CE02D0FFA3C080E10E946415892B09F4F9
:1008D0009DC0C1E0D1FF06C081E10E946415892B53
:1008E00009F096C0D2FF06C082E10E946415892BF0
:1008F00009F090C0D3FF06C083E10E946415892BE4
:1009000009F08AC0D4FF06C084E10E946415892BD7
:1009100009F084C0D5FF06C085E10E946415892BCB
:1009200009F07EC0D6FF06C086E10E946415892BBF
:1009300009F078C0D7FF06C087E10E946415892BB3
:1009400009F072C040E06C2F82E00E941903809190
:10095000F502882309F476C0D091CF02D0FF66C09B
:1009600088E10E946415892B09F460C0C1E0D1FFC1
:1009700006C089E10E946415892B09F059C0D2FF95
:1009800006C08AE10E946415892B09F053C0D3FF89
:1009900006C08BE10E946415892B09F04DC0D4FF7D
:1009A00006C08CE10E946415892B09F047C0D5FF71
:1009B00006C08DE10E946415892B09F041C040E01A
:1009C0006C2F83E0DF91CF910C941903C0E0E8CE47
:1009D000C260EECEC460F4CEC860FACEC06100CF73
:1009E000C06206CFC0640CCFC06812CFC0E025CF74
:1009F000C2602BCFC46031CFC86037CFC0613DCF5C
:100A0000C06243CFC06449CFC0684FCFC0E062CF5F
:100A1000C26068CFC4606ECFC86074CFC0617ACF47
:100A2000C06280CFC06486CFC0688CCFC0E09FCF4B
:100A3000C260A5CFC460ABCFC860B1CFC061B7CF33
:100A4000C062BDCFDF91CF910895109247028FEF22
:100A500080930A010895CF92DF92EF92FF920F9355
:100A60001F93CF93DF93182FEB01E82EF12CC701D2
:100A700080539D4F6C01FC0180818F3709F4EEC0DB
:100A8000863051F480914702882331F06630710539
:100A900009F4E0C00E9425051E31A8F4C430D10538
:100AA00091F0F701ED5FFD4F20812C3060F430E0D4
:100AB000C901880F991F820F931F8F5D9D4F0E9460
:100AC0003F0C8111B4C00EEE010F0C3058F461E000
:100AD00070E0C230D10511F060E070E0802F0E941C
:100AE000760202C01E31D0F4E12FE695E695E69538
:100AF000812F8770F0E0E453FD4F21E030E0082EB5
:100B000001C0220F0A94EAF7209721F48081822BFA
:100B1000808304C02095808128232083F701EE0F75
:100B2000FF1FE057FD4F11821082C230D10579F0CE
:100B30002CF42097C9F0219729F16BC0C430D1055E
:100B400009F445C064F1269709F45BC062C00C301B
:100B500008F084C060E0812F0E94F51460E0812FCE
:100B60000E942E1582E052C01E3108F077C060E06E
:100B7000812F0E94F51460E0812F0E942E15F6014E
:100B800010826CC01E3108F069C060E0812F0E94A5
:100B90002E1561E0812F0E94F51481E037C01330DB
:100BA00059F08BEF810F823038F087EF810F83305F
:100BB00018F01D3009F052C061E0812F0E94F51439
:100BC00060E070E0812F0E94211483E01FC01E317D
:100BD00008F044C084E0F6018083F701ED5FFD4F2B
:100BE00080818F3F41F190E09C01220F331F280F3D
:100BF000391FC9018F5D9D4F0E943F0C81112EC08E
:100C00001AC08EEF810F823048F586E0F6018083AE
:100C100025C06CE271E08EED93E0DF91CF911F91E2
:100C20000F91FF90EF90DF90CF900C943811812FAF
:100C30000E94ED0248CF4FEF5FEF6FEF7FEF812F04
:100C4000DF91CF911F910F91FF90EF90DF90CF90A8
:100C50000C94A7021E3108F424CF35CFDF91CF9139
:100C60001F910F91FF90EF90DF90CF900895CF9359
:100C7000C0E08EEF8C0F823028F466E070E08C2F9D
:100C80000E942B05CF5FCE31A1F781E08093470210
:100C90008EE193E0CF910C94E50C0F931F93CF93CB
:100CA000DF9381E08093F4018091470281110E94DB
:100CB0002505E2EFF2E0CCECD2E0AEEEB2E011922C
:100CC00019921D9282E0E63FF807C9F7C3E0D2E02F
:100CD00010E00FEF8EEE810F8C3018F462E070E0C0
:100CE00002C061E070E0812F0E942B0509931F5F15
:100CF0001E3181F71092F7021092F6021092F6015F
:100D00001092F5011092F401DF91CF911F910F9194
:100D1000089524E042E06DE371E08EED93E00E94DF
:100D2000D00F4BE352E060EE8EED93E00E9446114F
:100D300044EC51E060E98EED93E00E94461146E7F5
:100D400052E060EC8EED93E00E94461147E353E0E1
:100D500060ED8EED93E00E9446114BE255E064EFAA
:100D60008EED93E00E94461143E557E060EF8EED73
:100D700093E00E9471114DE456E06FEF8EED93E029
:100D80000E94691140E051EE60E070E08EED93E06A
:100D90000E94C9120C944D06CF93DF93C1E2D2E0BA
:100DA000CE010E94F90A239682E0C534D807C1F724
:100DB000DF91CF910895682F8EE193E00C94A60CFB
:100DC0008EE193E00E94560C0895DF92EF92FF921D
:100DD0000F931F93CF93DF93F82EEB01D42E6F3F29
:100DE0008FEF7807A9F06F2D8EE193E00E94FF0C42
:100DF0008C2F0E94DB068EE193E00E941C0D8091F7
:100E0000450290914602009729F00E948F1302C07C
:100E1000C0E0D0E04D2D6F2D8EE193E00E94FC0CE0
:100E20000D2D10E08EE193E00E944E0C081719077B
:100E30001CF461E571E009C08EE193E00E944E0C64
:100E40008017910734F46EE671E08EED93E00E9416
:100E50003811F0924802C09349028AE4E82E82E0F9
:100E6000F82EC0E0D0E0C017D10784F042E04D0D6D
:100E700028E432E067E78EED93E0DF91CF911F9198
:100E80000F91FF90EF90DF900C94F0108EE193E0C3
:100E90000E944E0C892B51F30E94E006F7018193CA
:100EA0007F012196E0CFEF92FF920F931F93CF9394
:100EB000DF93162FEA0190E0FC01E956F109E231D7
:100EC000F10508F03CC2EA5AFF4F0C94141D8981C9
:100ED000982F987185FF03C06AE871E056C0888139
:100EE000983071F148F491112AC2682F8EE193E095
:100EF0000E94FF0C02E007C0903109F440C0983115
:100F000009F471C01CC2011768F4FE01E00FF11D65
:100F10009181808120E8929F801911240E94DB0634
:100F20000E5FF1CF8EE193E00E941C0D86E490E00D
:100F3000DF91CF911F910F91FF90EF900C948F1341
:100F40004A816B81163069F430E8639FB001112447
:100F5000640F711D9D814C8150E8959F40191124AB
:100F600006C090E8699F401911246FEF7FEFDF9171
:100F7000CF911F910F91FF90EF900C94E506E091B7
:100F80000A01E73064F06AEA71E08EED93E0DF91E8
:100F9000CF911F910F91FF90EF900C9438119A818F
:100FA0002B81F0E8663061F42F9F90011124290F06
:100FB000311D4D819C8150E8459F9019112405C039
:100FC0002F9F901911242FEF3FEFEF5FE0930A015D
:100FD00044E0E402F0011124E859FD4F808332839C
:100FE00021839383ACC150910A01151634F440E07B
:100FF000252F332727FD30950EC08FEF80930A01F0
:101000009EC1EE0FFF1FEE0FFF1FE859FD4F9081AD
:10101000981719F14F5FE42FF0E02E173F078CF778
:1010200040E01BC04830C0F4DF01AA0FBB1FAA0F6D
:10103000BB1FA459BD4F8C91EE0FFF1FEE0FFF1F7A
:10104000E859FD4F808311968D919C911297928360
:10105000818313968C9183834F5FE42FF0E02E17EA
:101060003F0704F7515050930A0169C128818981D3
:1010700050E8859FC0011124820F911D009721F037
:10108000909346028093450280914702811157C197
:10109000DF91CF911F910F91FF90EF900C94370645
:1010A000653008F44CC118810981FA80EB80CC814D
:1010B0001E3108F044C1E12FF0E0ED5FFD4FE0810B
:1010C000EC3060F4F0E0CF01880F991F8E0F9F1F66
:1010D0008F5D9D4F0E943F0C81112DC180E8C89FFC
:1010E000A00111244E0D511D90E8F99EB00111246C
:1010F000600F711D812F0E94A70264E070E0812FB4
:10110000DF91CF911F910F91FF90EF900C942B05E1
:10111000623008F414C128818981E0E88E9FC00103
:101120001124820F911D90930C0180930B010A975B
:1011300008F005C18AE090E090930C0180930B01C8
:10114000FEC0623008F4FBC0698170E0123091F09B
:101150008A81F0E88F9FC0011124682B792B13300E
:1011600049F08B8190E090E4899F902D882711248D
:10117000682B792B8881DF91CF911F910F91FF9080
:10118000EF900C943B0260EF8EED93E00E943C11D7
:101190006CE68EED93E00E943C11C0E060E08EEDC5
:1011A00093E00E943C1161E08EED93E00E943C11BF
:1011B00061E08EED93E00E943C1161E08EED93E0E2
:1011C0000E943C118EEE8C0F8C3058F462E08EED54
:1011D00093E00E943C116AE08EED93E00E943C1186
:1011E0000DC0C33059F463E08EED93E00E943C11D2
:1011F00068E08EED93E00E943C110AC08BEF8C0FEB
:10120000823088F387EF8C0F833068F3CD3059F349
:1012100064E08EED93E00E943C116EE08EED93E071
:101220000E943C118EEF8C0F823050F466E08EED00
:1012300093E00E943C1161E08EED93E00E943C112E
:101240006FE78EED93E00E943C11CF5FCE3109F045
:10125000A5CF67EF8EED93E0DF91CF911F910F91B6
:10126000FF90EF900C943C11662309F468C0C8818C
:1012700060EF8EED93E00E943C116EE68EED93E000
:101280000E943C116C2F8EED93E00E943C11CE31F8
:1012900000F7D0E0FE01E053FD4F60818EED93E05A
:1012A0000E943C11CC0FDD1F8E0100571D4FF8012D
:1012B00060816F778EED93E00E943C11F8016081B0
:1012C0007181CB018078892B49F0660F672F661FEB
:1012D000770B6F778EED93E00E943C11C057DD4F86
:1012E00068817981CB018827907C892B09F4B1CF63
:1012F000770F660B770F762F661F6F778EED93E073
:101300000E943C11A6CF60EF8EED93E00E943C114D
:101310006AE68EED93E00E943C11CEEECC3010F0E8
:101320006FE701C06C2F8EED93E00E943C11CF5F00
:10133000CC30A1F78ECF812F0E94ED02CFCEDF916E
:10134000CF911F910F91FF90EF9008958F929F92F0
:10135000AF92BF92CF92DF92EF92FF920F931F93C3
:10136000CF93DF930E94BE038EED93E00E94301076
:10137000892B29F08EED93E00E949C11F5CF0E94FD
:10138000381360938C0270938D0280938E02909339
:101390008F02C0908802D0908902E0908A02F0907B
:1013A0008B0240910B0150910C014A01A12CB12CF0
:1013B0008B019C010C191D092E093F09801691060D
:1013C000A206B30608F04CC0D501C4018C0D9D1DCA
:1013D000AE1DBF1D8093880290938902A0938A025C
:1013E000B0938B02C0EDD2E01EEE1C30C0F48881B9
:1013F0008230A9F42091F6023091F702012E02C04A
:10140000359527950A94E2F720FF09C0812F0E94A5
:10141000F013AC01612F8EED93E00E94A9101F5FC5
:1014200021961C3011F780910A0187FD19C0C0E098
:10143000EC2FF0E080910A01992787FD90958E1797
:101440009F0774F0EE0FFF1FEE0FFF1FE859FD4FCF
:1014500061817281438180810E94E506CF5FE8CF80
:10146000DF91CF911F910F91FF90EF90DF90CF9080
:10147000BF90AF909F908F9008951F920F920FB6DC
:101480000F9211242F933F934F935F936F937F930A
:101490008F939F93AF93BF93EF93FF938091F90244
:1014A00087FF05C010928500109284001AC0209119
:1014B000F902332727FD30958091F80290E0281734
:1014C00039077CF48091F902992787FD9095FC01FA
:1014D000EE0FFF1FE80FF91FE650FD4F808186FDDC
:1014E00015C08091F9028F5F8093F9022091F90273
:1014F000332727FD30958091F80290E028173907AF
:10150000BCF48091F9028C305CF112C08091F90238
:10151000992787FD9095FC01EE0FFF1FE80FF91F3B
:10152000E650FD4F808160E08F730E942E15D9CF69
:101530008091840090918500049680349C4918F431
:1015400080E49CE905C08091840090918500049618
:1015500090938900809388008FEF8093F90238C0C0
:1015600020918400309185008091F902992787FDB0
:101570009095FC01EE0FFF1FE80FF91FE650FD4F9D
:1015800081819281820F931F9093890080938800BC
:101590008091F902992787FD9095FC01EE0FFF1FBE
:1015A000E80FF91FE650FD4F808186FF11C0809142
:1015B000F902992787FD9095FC01EE0FFF1FE80FB8
:1015C000F91FE650FD4F808161E08F730E942E1558
:1015D000FF91EF91BF91AF919F918F917F916F910B
:1015E0005F914F913F912F910F900FBE0F901F90E1
:1015F00018952091F8022C30A0F431E0320F30938E
:10160000F802FC012083822F90E0FC01EE0FFF1F07
:10161000E80FF91FE650FD4F88EB9BE09283818332
:1016200008952FEFFC0120830895DF92EF92FF923F
:101630000F931F93CF93DF93EC01D62E7A0189018C
:1016400088818C3008F066C061E08D2D0E94F51411
:101650008881A82FB0E0FD01EE0FFF1FEA0FFB1FEE
:10166000E650FD4F2D2D2F739081907C922B90830F
:1016700060E272E06E197F0977FF02C06D5F7F4FF5
:101680007595679575956795698340E659E0401BA8
:10169000510B57FF02C04D5F5F4F559547955595CC
:1016A00047954A836CE00E94C71C9CE0899FB0016B
:1016B000112420E030E0A901460F571FFA01EE0F78
:1016C000FF1FE40FF51FE650FD4F908196FD16C0F9
:1016D0002F5F3F4F2C30310571F781110FC01092F1
:1016E000800082E080938100109285001092840037
:1016F000B19A80916F00826080936F00888190E042
:10170000FC01EE0FFF1FE80FF91FE650FD4F80812F
:10171000806480838881DF91CF911F910F91FF902A
:10172000EF90DF90089520E639E040E252E00C941B
:10173000150BFC01808190E0FC01EE0FFF1FE80F0C
:10174000F91FE650FD4F80818F7B80830895FC0157
:1017500080818C3070F5918128E830E0291B3109B7
:1017600097FD3395220F331F220F331F6217730724
:101770007CF0928128E532E0291B310997FD3395F1
:10178000220F331F220F331F621773070CF49B01C4
:1017900022503109220F331F4FB7F89490E0FC011B
:1017A000EE0FFF1FE80FF91FE650FD4F3283218334
:1017B0004FBF08954F925F926F927F92AF92BF9208
:1017C000CF92DF92EF92FF920F931F93CF93DF930D
:1017D000EC01603282E078070CF040C077FD06C073
:1017E000653B71052CF064EB70E002C060E070E0D6
:1017F000898128E830E0281B310987FD3395220FC5
:10180000331F220F331F5901CC24B7FCC094DC2CAA
:10181000882777FD8095982F2A8148E552E0421B62
:10182000510927FD5395440F551F440F551F2A0199
:10183000662457FC6094762C7F926F925F924F9251
:1018400014EBE12EF12C00E010E020E030E0A901E3
:101850000E942C1B0F900F900F900F90CE01DF91E4
:10186000CF911F910F91FF90EF90DF90CF90BF909D
:10187000AF907F906F905F904F900C94A70BFC01FE
:10188000808190E0FC01EE0FFF1FE80FF91FE6508A
:10189000FD4F808186FB882780F9089580914E0353
:1018A00090E020914F03821B9109089520914F03EE
:1018B00080914E03281750F4E22FF0E0E05BFC4FDC
:1018C000808190E02F5F20934F0308958FEF9FEF6B
:1018D0000895E0914F0380914E03E81730F4F0E053
:1018E000E05BFC4F808190E008958FEF9FEF0895BB
:1018F0000895CF92DF92EF92FF920F931F93CF93B1
:10190000DF937C01CB018A0120912A03222389F0F5
:10191000EB016B01C40ED51ECC15DD0569F0699194
:10192000D701ED91FC910190F081E02DC70109955F
:10193000F3CF642F0E94D80DC801DF91CF911F9182
:101940000F91FF90EF90DF90CF900895CF93DF93AA
:101950001F92CDB7DEB7698320912A032223D1F0ED
:1019600020912B03203240F021E030E0FC01338352
:10197000228380E090E015C080912C03E82FF0E0F6
:10198000E35DFC4F998190838F5F80932C0380935C
:101990002B0305C061E0CE0101960E94D80D81E0C5
:1019A00090E00F90DF91CF910895FC011382128295
:1019B00048EE53E060E070E04483558366837783AC
:1019C0008FEB91E091838083089510924F031092E2
:1019D0004E0310922C0310922B030C94230D862F90
:1019E000413208F040E260E573E00E94410D109240
:1019F0004F0380934E03089521E00C94EF0C81E097
:101A000080932A0360934D0310922C0310922B03B2
:101A100008950F93062F21E040912B036DE273E0B0
:101A200080914D030E94850D10922C0310922B0380
:101A300010922A030F91089561E00C94090D8EE134
:101A400093E00C94D50C1092DD0381E08093DB03CE
:101A50001092DA0361E082E00E942E1561E083E0DB
:101A60000E942E15E9EBF0E080818E7F80838081DB
:101A70008D7F808388E48093B80085E48093BC00E8
:101A80000895413208F03FC09091DD039111FCCFE1
:101A900091E09093DD032093DB032FEF20937003FD
:101AA0001092B503240F2093B4039093DC0390911C
:101AB000DC03880F892B8093DC038091DA0381306B
:101AC00041F41092DA038091DC038093BB0085EC33
:101AD00001C085EE8093BC008091DD038130E1F38D
:101AE0008091B503841710F44091B50326EB33E0E1
:101AF000FB01D9018A2F821B841718F48D918193E1
:101B0000F9CF842F089580E008950F93413208F0B3
:101B100046C09091DD039111FCCF92E09093DD03DC
:101B20000093DB039FEF909370031092B5034093F3
:101B3000B403FB0166EB73E0DB019A2F961B94174D
:101B400018F491919D93F9CF1092DC039091DC03EE
:101B5000880F892B8093DC038091DA03813041F474
:101B60001092DA038091DC038093BB0085EC01C006
:101B700085EE8093BC00222321F08091DD0382302A
:101B8000E1F3809170038F3F61F0809170038032A8
:101B900051F080917003803341F483E007C081E00D
:101BA00005C080E003C082E001C084E00F91089589
:101BB000613298F42091DD03243089F4609392031C
:101BC000FC0184E993E0DC012A2F281B261718F476
:101BD00021912D93F9CF80E0089581E0089582E06E
:101BE000089585ED8093BC008091BC0084FDFCCFFE
:101BF0001092DD03089585EC8093BC001092DD0304
:101C000008951F920F920FB60F9211242F933F93B6
:101C10004F935F936F937F938F939F93AF93BF93F4
:101C2000EF93FF938091B900887F803609F49CC0C0
:101C300068F5883209F45BC090F4803109F454C02F
:101C400038F4882309F4F5C0883009F44DC0F5C094
:101C5000883109F44CC0803209F45DC0EEC0803494
:101C600009F468C048F4803309F455C0883309F09A
:101C7000E4C080937003A8C0803509F44FC0883554
:101C800009F45DC0883409F0D8C0D5C0883909F49A
:101C9000C6C0A8F4883709F467C038F4883609F458
:101CA00063C0803709F460C0C8C0883809F4B7C081
:101CB000803909F45FC0803809F0BFC05BC0803B49
:101CC00009F485C038F4803A09F466C0883A09F40A
:101CD0007EC0B3C0803C09F4A6C0883C09F4A3C010
:101CE000883B09F489C0A9C08091DC0310C09091A1
:101CF000B5038091B403981770F5E091B50381E0C6
:101D00008E0F8093B503F0E0EA54FC4F80818093FE
:101D1000BB0085EC85C0809370038DC0E091B50356
:101D200081E08E0F8093B5038091BB00F0E0EA5410
:101D3000FC4F80839091B5038091B4036DC0E09116
:101D4000B50381E08E0F8093B5038091BB00F0E076
:101D5000EA54FC4F80838091DB0381116CC081E0E9
:101D60008093DA0384EA60C083E08093DD031092FD
:101D70007103CFCF80917103803208F050C0E091A1
:101D8000710381E08E0F809371038091BB00F0E0BE
:101D9000EE58FC4F8083BDCF80917103803230F4C8
:101DA000E0917103F0E0EE58FC4F10820E94F10DBB
:101DB0006091710370E0E091D603F091D70382E760
:101DC00093E00995109271030E94FB0D36C084E0E8
:101DD0008093DD031092930310929203E091D80355
:101DE000F091D903099580919203811105C081E09A
:101DF0008093920310929403E091930381E08E0FFD
:101E000080939303F0E0EC56FC4F80818093BB00FD
:101E10009091930380919203981708F47ACF85E804
:101E20008093BC000AC085EC8093BC001092DD0357
:101E300004C0109270030E94F10DFF91EF91BF91C9
:101E4000AF919F918F917F916F915F914F913F9152
:101E50002F910F900FBE0F901F9018950F931F9307
:101E6000CF93DF93EC018B0188819981DC01ED91A7
:101E7000FC916F770190F081E02D0995888199811F
:101E8000DC01ED91FC91B801660F672F661F770B9F
:101E90006F770190F081E02DDF91CF911F910F912D
:101EA0000994DC018D919C91DC01ED91FC910190F4
:101EB000F081E02D60EF0994DC018D919C91DC01B3
:101EC000ED91FC910190F081E02D67EF0994CF93A3
:101ED000DF93EC0188819981DC01ED91FC91019007
:101EE000F081E02D69EF099588819981DC01ED9100
:101EF000FC910190F081E02D62E009958881998143
:101F0000DC01ED91FC910190F081E02D64E0DF9126
:101F1000CF9109941F93CF93DF93EC018A8188239B
:101F2000D9F1CE010E94510F88819981DC01ED9198
:101F3000FC910190F081E02D69E7099588819981F4
:101F4000DC01ED91FC91AB81BC810190F081E02D31
:101F50006C91099588819981DC01ED91FC91AB81AF
:101F6000BC810190F081E02D11966C91099512E0F1
:101F70008A81181758F4EB81FC81E10FF11D608113
:101F800070E0CE010E942E0F1F5FF2CFCE01DF91D5
:101F9000CF911F910C945C0FDF91CF911F91089509
:101FA000CF92DF92EF92FF920F931F93CF93DF9325
:101FB0008C01EB01C42ED22E6BEC71E0CE010E949D
:101FC000751E7C016FE270E0CE010E946A1E0097D0
:101FD00039F46CE570E0CE010E946A1E009711F0A2
:101FE000EC012196E114F10451F4FE01019000206E
:101FF000E9F7EC1BEF5FD8011296EC9306C0EC1AE0
:10200000FD0AE394E394F801E282D80113968D91DE
:102010009C9114970E94CC1DF801E280F12CC7011D
:1020200001960E94341DD80114969C938E931397A9
:10203000FC01EE0DFF1D1082FC01C082D1821296C0
:102040004C9150E042505109BE010296DF91CF9170
:102050001F910F91FF90EF90DF90CF900C945B1E3B
:10206000DC018D919C91DC01ED91FC910480F58166
:10207000E02D09940F931F93CF93DF93FC012085EC
:10208000213749F0293709F049C0DF91CF911F91DD
:102090000F910C948A0FFC01E95AFF4F0190F081D7
:1020A000E02D309709F450C0DC01A75BBF4F4D9184
:1020B0005C919A012150310937FD9A01B90175955A
:1020C0006795062F40E050E020E030E04E5F5F4F24
:1020D0002017A0F4EC01C40FD51F1F81DC01A20F53
:1020E000B31F18961C931897C885D0E8CD9F101978
:1020F000112418961C932F5F3F4FE8CFDC01A60FE9
:10210000B11D17962C911797222311F018961C9247
:102110000896DF91CF911F910F910994FC01E75A26
:10212000FF4F0190F081E02D309771F0AC01475FD7
:102130005F4FDC01A75BBF4F6C916150822FDF9135
:10214000CF911F910F910994DF91CF911F910F9122
:1021500008950F931F93CF93DF93EC018A01888139
:102160009981DC01ED91FC916F70606E0190F081BE
:10217000E02D0995B801CE01DF91CF911F910F910C
:102180000C942E0F0F931F93CF93DF93EC018A01D2
:1021900088819981DC01ED91FC916F7060690190FB
:1021A000F081E02D099588819981DC01ED91FC9108
:1021B000602F6F770190F081E02D099588819981DA
:1021C000DC01ED91FC91B801660F672F661F770B5C
:1021D0000190F081E02DDF91CF911F910F91099433
:1021E000CF92DF92EF92FF920F931F93CF93DF93E3
:1021F00000D01F92CDB7DEB78C01F42E2A833B832B
:1022000069830E94510FD8018D919C91DC01ED9161
:10221000FC910190F081E02D698109952A81E22EDF
:10222000C22E3B81D32E8C2D8E198F1540F4F601D2
:1022300061916F0170E0C8010E942E0FF4CFC801B8
:102240000F900F900F90DF91CF911F910F91FF9002
:10225000EF90DF90CF900C945C0F9A01FA010190FF
:102260000020E9F73197E41BF50B4E2F0C94F0108A
:10227000AB0161E70C942D11DC018D919C91DC0187
:10228000ED91FC910190F081E02D0994603DB9F051
:1022900028F4603961F0603C71F00895603E19F0F7
:1022A000643F89F00895FC01E55BFF4F0FC0FC011E
:1022B000E35BFF4F0BC0FC01E15BFF4F07C0FC017C
:1022C000EF5AFF4F03C0FC01ED5AFF4F518340838B
:1022D00008956F3F29F4FC01EB5AFF4F518340836F
:1022E0000895875A9F4FFC01518340830895FC0154
:1022F00015821682178280E090E0DF01A80FB91FD7
:1023000018961C92019680349105B9F7DF01A85BFD
:10231000BF4F1C9211961D921C92EB5AFF4F0190D9
:10232000F081E02D309709F009940895FC011282A4
:10233000148213820C947711CF93DF93EC01888180
:102340009981DC01ED91FC910680F781E02D0995E2
:10235000FE01E85BFF4F20812223B1F0873F91050A
:1023600031F41082CE01DF91CF910C943A10FE012E
:10237000E75BFF4F20813181C20FD31F88872F5F1A
:102380003F4F318320839DC02D81222309F45EC0FD
:10239000803891050CF05AC09FEF920F9D83FE018B
:1023A000E90FF11D808791118CC08E81882309F47B
:1023B00088C0803DE9F148F48039E9F0803C09F0BB
:1023C00043C0FE01E15BFF4F36C0803E19F0843F01
:1023D00019F13AC0FE01E55BFF4F0190F081E02D5D
:1023E000309791F18885698570E0B0E88B9F600D2A
:1023F000711D112427C0FE01E35BFF4F0190F081A6
:10240000E02D309709F18885698570E090E8899F13
:10241000600D711D112416C0FE01ED5AFF4F019091
:10242000F081E02D309781F0688570E089850BC0E0
:10243000FE01EF5AFF4F0190F081E02D309721F01F
:10244000688570E08F8109951E823BC0803F9105B1
:102450002CF4282F2F702F83807F9927803E9105A1
:1024600021F154F4803C910511F1803D9105F9F082
:102470008039910531F519C0843F9105B1F054F4CC
:10248000803F9105F1F481E08083C75BDF4F1982C3
:10249000188217C0893F910571F08F3F910589F42B
:1024A000CE01DF91CF910C94771192E001C091E0C1
:1024B0009D838E8306C08EED93E0DF91CF910C94C7
:1024C000670FDF91CF9108958F929F92AF92BF9245
:1024D000CF92DF92EF92FF921F93CF93DF93EB01A6
:1024E0004A01690161E08DE00E94F51410E0EE24DC
:1024F000D7FCE094FE2CAA2497FCA094BA2C812F40
:1025000090E08C179D0794F4C701B6010E946713F1
:1025100061E08DE00E942E15C501B4010E94671391
:1025200060E08DE00E942E151F5FE9CFDF91CF9113
:102530001F91FF90EF90DF90CF90BF90AF909F9052
:102540008F900895CF93DF93EC0161E08DE00E94BE
:10255000F51422ED30E048E250E062E070E0CE0198
:102560000E9464126AEF70E080E090E00E946713BE
:1025700022ED30E048E250E064E070E0CE010E94DD
:1025800064126DE770E080E090E0DF91CF910C94F1
:102590006713CF93DF93EC0188E494E00E944A161E
:1025A00088E494E099838883CE010E94A212CE0130
:1025B0000E94670FCE01DF91CF910C948A0F8EEDB0
:1025C00093E00C9496110F9300E020E040E060E06F
:1025D00089E394E00E94A7160F9108951F920F922D
:1025E0000FB60F9211242F933F938F939F93AF9326
:1025F000BF938091400490914104A0914204B09116
:10260000430430913F0423E0230F2D3720F401963B
:10261000A11DB11D05C026E8230F0296A11DB11D05
:1026200020933F048093400490934104A09342047C
:10263000B09343048091440490914504A0914604D2
:10264000B09147040196A11DB11D8093440490935D
:102650004504A0934604B0934704BF91AF919F9166
:102660008F913F912F910F900FBE0F901F90189553
:102670002FB7F89460914004709141048091420416
:10268000909143042FBF08953FB7F894809144047C
:1026900090914504A0914604B091470426B5A89BAB
:1026A00005C02F3F19F00196A11DB11D3FBF662740
:1026B000782F892F9A2F620F711D811D911D42E085
:1026C000660F771F881F991F4A95D1F70895CF92FB
:1026D000DF92EF92FF92CF93DF936B017C010E9418
:1026E0004413EB01C114D104E104F10489F00E9408
:1026F000731B0E9444136C1B7D0B683E734090F368
:1027000081E0C81AD108E108F108C851DC4FEACFCE
:10271000DF91CF91FF90EF90DF90CF9008958230BE
:10272000910538F0880F991F880F991F0597019719
:10273000F1F70895789484B5826084BD84B5816092
:1027400084BD85B5826085BD85B5816085BDEEE6B9
:10275000F0E0808181608083E1E8F0E01082808198
:1027600082608083808181608083E0E8F0E0808106
:1027700081608083E1E9F0E08081826080838081F4
:1027800081608083E0E9F0E0808181608083E1EC1A
:10279000F0E080818460808380818260808380819A
:1027A00081608083E3ECF0E0808181608083E0ECF5
:1027B000F0E0808182608083E2ECF0E080818160E3
:1027C0008083EAE7F0E0808184608083808182609A
:1027D0008083808181608083808180688083089588
:1027E000823108F08251E82FF0E0E45FFE4FE4917F
:1027F00080917B00E3FB222720F930E095E0220F57
:10280000331F9A95E1F78F7D822B80937B00E770D1
:1028100080910D0120E4829FC0011124E82BE093F8
:102820007C0080917A00806480937A0080917A00A5
:1028300086FDFCCF809178002091790090E0922B6A
:1028400008951F93CF93DF93182FEB0161E00E944F
:10285000F514209711F460E004C0CF3FD10539F49E
:1028600061E0812FDF91CF911F910C942E15E12F04
:10287000F0E0E85EFE4F449150E0FA013197EF300E
:10288000F10508F06CC0E859FF4F0C94141D84B595
:10289000806884BDC7BD68C084B5806284BDC8BD82
:1028A00063C080918000806880938000D09389000D
:1028B000C093880059C0809180008062809380001E
:1028C000D0938B00C0938A004FC0809180008860B5
:1028D00080938000D0938D00C0938C0045C0809180
:1028E0009000806880939000D0939900C0939800E6
:1028F0003BC080919000806280939000D0939B00B9
:10290000C0939A0031C080919000886080939000BD
:10291000D0939D00C0939C0027C08091C000806828
:102920008093C0008091C0008F7B8093C000C093D3
:10293000CF001AC08091C00080628093C000C09315
:10294000D00012C08091C20088608093C200809144
:10295000C2008B7F8093C200C093D20005C0C038F4
:10296000D1050CF07DCF77CFDF91CF911F910895E6
:1029700090E0FC013197EF30F105B0F5E958FF4FD9
:102980000C94141D809180008F7703C0809180008B
:102990008F7D80938000089580918000877FF9CF9C
:1029A00084B58F7702C084B58F7D84BD08958091F2
:1029B00090008F7707C0809190008F7D03C0809139
:1029C0009000877F8093900008958091C0008F775A
:1029D00003C08091C0008F7D8093C00008958091D6
:1029E000C200877F8093C2000895CF93DF9390E069
:1029F000FC01EA5CFE4F2491FC01EC5AFE4F8491ED
:102A0000882349F190E0880F991FFC01E257FE4F9F
:102A1000A591B49180589E4FFC01C591D4919FB768
:102A2000611108C0F8948C91209582238C93888141
:102A300082230AC0623051F4F8948C91322F309581
:102A400083238C938881822B888304C0F8948C9193
:102A5000822B8C939FBFDF91CF9108950F931F938B
:102A6000CF93DF931F92CDB7DEB7282F30E0F90167
:102A7000E85EFE4F8491F901EA5CFE4F1491F90182
:102A8000EC5AFE4F04910023C9F0882321F069839A
:102A90000E94B8146981E02FF0E0EE0FFF1FE058AC
:102AA000FE4FA591B4919FB7F8948C91611103C02A
:102AB0001095812301C0812B8C939FBF0F90DF91D4
:102AC000CF911F910F910895CF93DF93282F30E07E
:102AD000F901E85EFE4F8491F901EA5CFE4FD49162
:102AE000F901EC5AFE4FC491CC2391F081110E9460
:102AF000B814EC2FF0E0EE0FFF1FEE58FE4FA5913B
:102B0000B4912C912D2381E090E021F480E002C06B
:102B100080E090E0DF91CF910895CF93DF931F92F3
:102B2000CDB7DEB76983DC01ED91FC910280F381C2
:102B3000E02D41E050E0BE016F5F7F4F09950F909F
:102B4000DF91CF910895CF93DF93EC018C859D8524
:102B500097FF05C082E00E9459189D878C878C855D
:102B60009D85DF91CF91089583E00C94AE1AFC010E
:102B70008485958597FD06C082E00E94011890E04B
:102B80000196089582E00E94011890E00895FC01EA
:102B90008485958597FD05C02FEF3FEF3587248706
:102BA000089582E00C945918CF93DF93EC01809143
:102BB0001501882331F083E00E948A18181619063F
:102BC00034F081E090E09B838A8380E090E0DF91A5
:102BD000CF910895FC0120812E5F208342E450E0D4
:102BE0006CE971E080E80C942519FC0181819081E9
:102BF000913A59F4813209F03CC047E050E06EE070
:102C000071E080E00E94251943C0913291F5803235
:102C100039F467E070E08EE091E00E94561906C03A
:102C2000823209F035C082818093150180910E01B6
:102C300090910F01A0911001B0911101803B94403F
:102C4000A105B105C1F48091150180FD14C087E78D
:102C500097E790930108809300082BE088E190E0CB
:102C60000FB6F894A895809360000FBE2093600083
:102C70000FC080E0089588E10FB6F894809360005B
:102C8000109260000FBEA8951092010810920008E3
:102C900081E008952FEF3FEFFC01358724870895E9
:102CA00010924B0410924A0488EE93E0A0E0B0E04A
:102CB00080934C0490934D04A0934E04B0934F0422
:102CC00084ED91E090934904809348048FEF9FEF47
:102CD00090935504809354040895AF92BF92CF927D
:102CE000DF92EF92FF920F931F93CF93DF936C01CC
:102CF0007B01C0E0D0E000E010E0F601EC0FFD1F2A
:102D00004AE050E06281C7010E9481175C016EE2D7
:102D1000C7010E9414178A0D9B1D080F191F2196C9
:102D2000C330D10551F74AE050E0F6016581C70193
:102D30000E948117800F911FDF91CF911F910F91FA
:102D4000FF90EF90DF90CF90BF90AF9008950F93DA
:102D5000FC0184EE91E0918380836283438324832A
:102D600005830F91089584EE91E0909399048093E8
:102D7000980410929A0410929B0410929C04109252
:102D80009D04089508950E949A130E94C2168EE928
:102D900094E00E940E1B0E948906C0E0D0E00E94D1
:102DA000A6092097E1F30E940000F9CFCF92DF92AD
:102DB000EF92FF920F931F93CF93DF936C017A01F1
:102DC000EB01E60EF71E00E010E0CE15DF0561F026
:102DD0006991D601ED91FC910190F081E02DC60141
:102DE0000995080F191FF1CFC801DF91CF911F91ED
:102DF0000F91FF90EF90DF90CF90089561157105CE
:102E000081F0DB010D900020E9F7AD01415051093F
:102E1000461B570BDC01ED91FC910280F381E02D04
:102E2000099480E090E00895DC01ED91FC9101901F
:102E3000F081E02D09948F929F92AF92BF92CF9232
:102E4000DF92EF92FF920F931F93CF93DF93CDB753
:102E5000DEB7A1970FB6F894DEBF0FBECDBF7C01E1
:102E6000C42EE52FCB01D22E19A221E02D1510F092
:102E70002AE0D22E8E010F5D1F4F8D2C912CA12C9C
:102E8000B12C6C2D7E2FA50194010E94D31C8C2D9A
:102E9000D29E80191124015011098A3014F4805DEA
:102EA00001C0895CF8018083211531054105510578
:102EB00021F0C22EE32FCA01E4CFB801C7010E945E
:102EC000FE16A1960FB6F894DEBF0FBECDBFDF9100
:102ED000CF911F910F91FF90EF90DF90CF90BF9017
:102EE000AF909F908F9008952115310541F4DC013A
:102EF000ED91FC910190F081E02D642F09940C94E8
:102F00001B179A01462F50E060E070E00C94741794
:102F10004091A2045091A3042091A0043091A104F7
:102F200042175307B4F49091E8009570E1F3909143
:102F3000E80092FD19C08093F1008091A204909165
:102F4000A30401968F739927892B19F48EEF809330
:102F5000E8008091A2049091A30401969093A304A9
:102F60008093A20481E0089580E00895CF92DF92DB
:102F7000FF920F931F93CF93DF931F92CDB7DEB7CE
:102F8000082F162F862F880F8E5F99830E9488172F
:102F900083E00E948817F02EC02E9981D92E8C2DA7
:102FA0008F19811778F4F60184910E948817082FF1
:102FB00080E00E9488178023FFEFCF1ADF0A81117B
:102FC000EECF01C081E00F90DF91CF911F910F9163
:102FD000FF90DF90CF900895615030F02091F10084
:102FE000FC0120830196F8CF289884E68093A504FD
:102FF00008952FB7FC012083F89467706093E9006F
:103000000895CF93DF931F92CDB7DEB7682FCE011F
:1030100001960E94F9178091F20099819FBF0F904D
:10302000DF91CF910895FF920F931F93CF93DF937A
:1030300000D0CDB7DEB7F62E8A019091A404992373
:1030400011F057FF03C08FEF9FEF2BC0682FCE0109
:1030500001967A830E94F9178091F20090E0A8010E
:103060007A81801791070CF4AC01EF2DF72FF40E45
:1030700084E6FE1639F028988093A5049091F1001B
:103080009193F7CF4115510521F08091F2008823EB
:1030900021F089818FBFCA0104C08BE68093E800CC
:1030A000F8CF0F900F90DF91CF911F910F91FF906C
:1030B0000895CF93DF931F92CDB7DEB741E050E084
:1030C000BE016F5F7F4F0E941318019719F4898129
:1030D00090E002C08FEF9FEF0F90DF91CF910895A6
:1030E000CF93DF931F92CDB7DEB7682FCE01019645
:1030F0000E94F9179091E800892F807295FF04C013
:103100009091F20080E4891B99819FBF0F90DF911D
:10311000CF9108956F927F928F929F92AF92BF92BC
:10312000CF92DF92EF92FF920F931F93CF93DF9393
:103130001F92CDB7DEB7782E7B01C42EB52E8091BD
:10314000A404882369F0042F152F8AEFD82E872D29
:103150008072982E9AE3A92E872D8074882E11C034
:103160008FEF9FEF57C0872D0E947018682E811136
:103170000CC0DA94A9F361E070E080E090E00E9476
:1031800067130115110579F73BC0282F30E00217AE
:1031900013070CF4602E672DCE0101960E94F917DB
:1031A0008091E80085FF29C0262D30E0021B130B1B
:1031B000992039F06A948FEF6816B1F01092F100FF
:1031C000F9CFF701862D77FE07C0815058F0949112
:1031D0009093F1003196F9CF815020F09191909326
:1031E000F100FACFE20EF31E8091E80085FF0FC0D8
:1031F0000115110511F481100AC089818FBFC1CF5B
:103200005D9884E68093A6048C2D9B2D03C0A0922C
:10321000E800F3CF0F90DF91CF911F910F91FF90B6
:10322000EF90DF90CF90BF90AF909F908F907F9066
:103230006F9008951092E9001092A3041092A204D6
:103240009093A1048093A0040895CF92DF92FF92FF
:103250000F931F93CF93DF9300D0CDB7DEB7F82E37
:103260008A016B0101151105B1F0F601F7FE02C0EC
:10327000849101C0808149835A830E94881701503C
:103280001109FFEFCF1ADF0A49815A818111EACF74
:103290008FEF9FEF01C0CA010F900F90DF91CF9188
:1032A0001F910F91FF90DF90CF9008951F93CF93C0
:1032B000DF931F92CDB7DEB7162F2091E80022FFD3
:1032C000FCCF612F79830E94EC178BEF8093E8008D
:1032D000812F7981972F0F90DF91CF911F910895C2
:1032E000CF93DF931F92CDB7DEB71982CE0101963F
:1032F0000E94EA15CE0101960E94921B898190E0FE
:103300000F90DF91CF9108951F920F920FB60F92F9
:103310001124EF92FF920F931F932F933F934F939C
:103320005F936F937F938F939F93AF93BF93EF932D
:10333000FF93CF93DF93CDB7DEB76297DEBFCDBFEC
:103340001092E9008091E80083FFEBC068E0CE01B5
:103350000A960E94EC1782EF8093E8009A8597FF07
:1033600005C08091E80080FFFCCF03C08EEF809302
:10337000E800892F807609F0B9C08B85811105C0DE
:103380001092F1001092F100C5C0282F2D7F21303E
:1033900009F4C0C0853049F48091E80080FFFCCF7B
:1033A0008C8580688093E300B5C0863009F076C0D4
:1033B0002D85E888F988223071F580E090E02A8B2D
:1033C0000E941A190E94701999E08E010F5F1F4F19
:1033D000F801392F11923A95E9F799832A892A83BE
:1033E00091E09E8390E898879AEF99872091A204B4
:1033F0003091A304275F3F4F3C832B838D83C7010C
:103400000E941A1949E050E0B80180E00E94251995
:103410000E9470197FC0C7012A8B0E941A192A893D
:10342000223241F482E290E00E949D1B892B09F038
:1034300071C074C0213069F488899989089711F4A2
:1034400020939F0480919F04811118C065EF71E063
:103450001AC0233009F062C08C85882391F0823035
:1034600021F460E183E192E006C0813009F056C0AA
:103470006BE087E092E00E94B6174AC063EE71E00D
:1034800002C064E272E06115710509F447C0FB01F6
:10349000449150E080E80E9425193CC0873009F42F
:1034A0003DC0883021F481E08093F10033C0893041
:1034B00089F5937099F5EFEDF1E081E021E096E375
:1034C0008093E9002093EB0034913093EC009093CB
:1034D000ED008F5F3196853099F78EE78093EA0093
:1034E0001092EA008C858093A40414C0888999897D
:1034F0000E941A198E85811105C0CE010A960E947C
:10350000F51506C0823051F4CE010A960E94C51B03
:10351000882321F08EEF8093E80003C081E280933E
:10352000EB0062960FB6F894DEBF0FBECDBFDF9101
:10353000CF91FF91EF91BF91AF919F918F917F912B
:103540006F915F914F913F912F911F910F91FF903C
:10355000EF900F900FBE0F901F9018958093E90089
:103560008091F200882319F08AE38093E80008959F
:103570001F920F920FB60F9211242F933F934F93E8
:103580005F936F937F938F939F93AF93BF93EF93CB
:10359000FF938091E1001092E10083FF0FC0109231
:1035A000E90091E09093EB001092EC0092E390938D
:1035B000ED001092A40498E09093F00082FF1DC0EB
:1035C00083E00E94AE1A8091A604882339F080918E
:1035D000A60481508093A604882369F08091A504F5
:1035E000882359F08091A50481508093A50481110E
:1035F00004C0289A02C05D9AF1CFFF91EF91BF916C
:10360000AF919F918F917F916F915F914F913F917A
:103610002F910F900FBE0F901F9018951092A40439
:1036200081E08093D70080EA8093D80082E189BD51
:1036300009B400FEFDCF61E070E080E090E00E9400
:10364000671380E98093D8008CE08093E2001092A9
:10365000E000559A209A08954F925F926F927F9260
:10366000AF92BF92CF92DF92EF92FF920F931F9390
:10367000CF93DF93CDB7DEB729013A01621B730BFD
:10368000840B950B29893A894B895C892A193B0956
:103690004C095D09298B3A8B4B8B5C8B9B01AC01F0
:1036A00069897A898B899C890E94B71CE418F5087E
:1036B00006091709A80197010E94F51C2A0D3B1D58
:1036C0004C1D5D1DCA01B901DF91CF911F910F9172
:1036D000FF90EF90DF90CF90BF90AF907F906F9072
:1036E0005F904F9008950895FF920F931F93CF938B
:1036F000DF93EC01F62EE881F9810480F581E02D5D
:1037000009958C01E881F9810680F781E02D6F2D04
:10371000CE010995C8019927DF91CF911F910F9193
:10372000FF900895FC0120812F5F208349E150E044
:1037300068EA72E080E80C94251945E650E061ECF7
:1037400072E080E80C942519EF92FF920F931F937B
:10375000CF93DF931F92CDB7DEB789838B017A01B8
:1037600041E050E0BE016F5F7F4F84E00E948A1805
:10377000A701B80184E40E948A180F90DF91CF91CD
:103780001F910F91FF90EF900895FC01918180812E
:10379000813A31F481E0913091F0933089F411C095
:1037A000813271F49B3021F482818093170105C02E
:1037B0009A3031F482818093160181E00895089552
:1037C00080E0089548E050E082E00C94A41BCF9381
:1037D000DF93DC01683818F0E8E7E60F25C0E62F34
:1037E000F0E067FF11C0E058F10981E090E001C00E
:1037F000880FEA95EAF714969C911497982B1496E3
:103800009C931497E0E010C0E85DFD4FE491EE2337
:1038100009F440C0E7FF08C014968C9114978260A9
:1038200014968C931497EF7716968C9116978E17A3
:1038300041F117968C9117978E1719F118968C9164
:1038400018978E17F1F019968C9119978E17C9F069
:103850001A968C911A978E17A1F01B968C911B9734
:103860008E1779F080E090E0ED01C80FD91F2E810E
:10387000211102C0EE8305C0019686309105A1F7A3
:1038800009C0BD016C5F7F4FCD010E94E21B81E04A
:1038900090E008C081E090E013969C938E9312977D
:1038A00080E090E0DF91CF910895683818F0E8E764
:1038B000E60F25C0E62FF0E067FF12C0E058F109DF
:1038C00021E030E001C0220FEA95EAF72095DC0103
:1038D00014963C911497322314963C93E0E00FC069
:1038E000E85DFD4FE491EE2329F1E7FF08C0DC011C
:1038F00014962C9114972D7F14962C93EF7720E03B
:1039000030E0EE2351F0DC01A20FB31F16964C916C
:1039100016974E1302C016961C922F5F3F4F26300B
:10392000310579F7BC016C5F7F4F0E94E21B81E09B
:1039300090E0089580E090E00895FC0116821782DF
:1039400010861186128613861482BC016C5F7F4F2D
:103950000C94E21B1092B3041092AA041092A904D2
:103960008AEE91E09093A8048093A7040895DB0168
:103970008F939F930E941A1DBF91AF91A29F800DBC
:10398000911DA39F900DB29F900D11240895991B36
:1039900079E004C0991F961708F0961B881F7A9546
:1039A000C9F780950895A1E21A2EAA1BBB1BFD0141
:1039B0000DC0AA1FBB1FEE1FFF1FA217B307E4070E
:1039C000F50720F0A21BB30BE40BF50B661F771F66
:1039D000881F991F1A9469F7609570958095909546
:1039E0009B01AC01BD01CF010895052E97FB1EF48C
:1039F00000940E940C1D57FD07D00E94D31C07FCA9
:103A000003D04EF40C940C1D5095409530952195A3
:103A10003F4F4F4F5F4F08959095809570956195FA
:103A20007F4F8F4F9F4F0895EE0FFF1F0590F4912A
:103A3000E02D09940E94251DA59F900DB49F900D27
:103A4000A49F800D911D11240895A29FB001B39FE2
:103A5000C001A39F700D811D1124911DB29F700D97
:103A6000811D1124911D0895CF93DF93823091051C
:103A700010F482E090E0E091B604F091B70420E009
:103A800030E0A0E0B0E0309739F140815181481733
:103A90005907B8F04817590771F48281938110973C
:103AA00029F013969C938E9312972CC09093B70491
:103AB0008093B60427C02115310531F04217530712
:103AC00018F0A901DB0101C0EF019A01BD01DF017E
:103AD0000280F381E02DD7CF21153105F9F0281BA5
:103AE000390B2430310580F48A819B816115710581
:103AF00021F0FB019383828304C09093B7048093E9
:103B0000B604FE01329644C0FE01E20FF31F81931A
:103B1000919322503109398328833AC02091B4040B
:103B20003091B504232B41F420910201309103011F
:103B30003093B5042093B404209100013091010129
:103B40002115310541F42DB73EB740910401509144
:103B50000501241B350BE091B404F091B504E21784
:103B6000F307A0F42E1B3F0B2817390778F0AC01A0
:103B70004E5F5F4F2417350748F04E0F5F1F50937D
:103B8000B5044093B4048193919302C0E0E0F0E067
:103B9000CF01DF91CF910895CF93DF93009709F480
:103BA00087C0FC01329713821282C091B604D09173
:103BB000B704209781F420813181280F391F80912B
:103BC000B4049091B5048217930779F5F093B50486
:103BD000E093B4046DC0DE0120E030E0AE17BF0713
:103BE00050F412964D915C9113979D01411551052A
:103BF00009F1DA01F3CFB383A28340815181840FAD
:103C0000951F8A179B0771F48D919C911197840FD2
:103C1000951F02969183808312968D919C911397A4
:103C2000938382832115310529F4F093B704E0933F
:103C3000B6043EC0D9011396FC93EE9312974D91B2
:103C40005D91A40FB51FEA17FB0779F4808191817C
:103C5000840F951F0296D90111969C938E938281B1
:103C6000938113969C938E931297E0E0F0E08A8103
:103C70009B81009719F0FE01EC01F9CFCE0102966D
:103C800028813981820F931F2091B4043091B504AB
:103C90002817390769F4309729F41092B704109265
:103CA000B60402C013821282D093B504C093B40448
:103CB000DF91CF910895FB01DC014150504048F065
:103CC00001900D920020C9F701C01D924150504053
:103CD000E0F70895FC0181E090E00190061609F4F8
:103CE000CF010020D1F701970895FB015191552391
:103CF000A9F0BF01DC014D9145174111E1F759F4DD
:103D0000CD010190002049F04D9140154111C9F3BA
:103D1000FB014111EFCF81E090E001970895F89405
:023D2000FFCFD3
:103D22000000B804800001000000FF13000100E160
:103D320000000000000001014D6178207365727679
:103D42006F7320617474616368656400556E6B6E95
:103D52006F776E2070696E206D6F646500537461B9
:103D62006E646172644669726D6174612E696E6F10
:103D7200004932433A20546F6F206D616E792062A0
:103D8200797465732072656365697665640049328A
:103D9200433A20546F6F20666577206279746573A9
:103DA2002072656365697665640031302D626974DD
:103DB2002061646472657373696E67206E6F74202C
:103DC200737570706F7274656400746F6F206D61CB
:103DD2006E7920717565726965730000000000A636
:103DE2000C790C4E0C560C690C780C2E637070001A
:103DF200000000008D15D415B715C715A315B4150D
:103E0200000000006D1600000000741BD616E71BB0
:043E1200551C9D1C82
:00000001FF
